:020000040000FA
:040000008BEF0AF088
:08000800056ED8CF06F0E0CF31
:1000100007F00001E9CF0DF0EACF08F0E1CF09F0D9
:10002000E2CF0AF0D9CF0BF0DACF0CF0F3CF14F017
:10003000F4CF15F0FACF16F000C00FF001C010F0A9
:1000400002C011F003C012F004C013F0F2AA2CEFAA
:1000500000F0F2B4C5EF01F00FC000F010C001F0E5
:1000600011C002F012C003F013C004F00E8E0DC0D8
:10007000E9FF08C0EAFF09C0E1FF0AC0E2FF0BC0C8
:10008000D9FF0CC0DAFF14C0F3FF15C0F4FF16C08F
:10009000FAFF055007C0E0FF06C0D8FF10000DAE04
:1000A00003D0F2CF0EF0F29EF76AC00FF66E000E8C
:1000B000F7220900F5500DAE02D00EBEF28E1200EE
:1000C00053EF6EF0000000000DAE03D0F2CF0EF043
:1000D000F29EF76AEA0FF66E000EF7220900F5505D
:1000E0000DAE02D00EBEF28E120053EF6EE800008D
:1000F00000000DAE03D0F2CF0EF0F29EF76A140F9F
:10010000F66E010EF7220900F5500DAE02D00EBEBC
:10011000F28E1200457869740000000003011B6B29
:100120001B51070815E31AAF03D093928A8202D0BD
:1001300093928A9200D000D093948A8400D000D009
:10014000D8901A3793948A9400D000D01B2BE8D70C
:1001500093928A8200D000D00001000C93968A9678
:10016000020E03011A6F0001D9DF15C31AF3D6DF9F
:1001700017C318F30301196B17C31AF30001CEDF7D
:1001800016C31AF3CBDF93968A86000C0301156B16
:10019000176B040E166F0001E1DF550E006E002E86
:1001A000FED70301156B176B166B0001D7DF938C1D
:1001B00081ACFDD7030E0301156F980E176F166BF8
:1001C0000001CCDF550E006E002EFED70301106B30
:1001D00019C00FF319C012F3116B036A19501111F2
:1001E000136F03501910146F0B0E156F14C317F310
:1001F00013C316F30001B2DF550E006E002EFED7BA
:10020000000C030EEA6E0F0EE96EEF500EE00C0EBE
:10021000016E006A002EFED7012EFBD7F70E006E8E
:10022000002EFED700D0EF2EF2D7000CF29CF29EEB
:10023000F2BEFDD7ABDF0301156B176B200E166FF7
:1002400000018CDF550E006E002EFED7C00EF2129C
:1002500003010A53D8B493D009532BE00B6B0B5115
:10026000070826E3036A0B51F2CF0FF3F29E000159
:1002700016DF03010FBFF28E0E6F93988A880C6B06
:100280000C51070811E30EAF03D093928A8202D07B
:1002900093928A92939A8A8AD8900E37939A8A9ADE
:1002A00093988A980C2BECD793928A820B2BD7D7F2
:1002B0002AD00B6B0B51070826E3036A0B51F2CFD0
:1002C0000FF3F29E000100DF03010FBFF28E0E6FED
:1002D00093988A880C6B0C51070811E30EAF03D07A
:1002E00093928A8202D093928A92939A8A8AD89021
:1002F0000E37939A8A9A93988A980C2BECD79392FC
:100300008A820B2BD7D7320E0F6F00017ADF0301E1
:100310000D6B0D5101082CE30B6B0B51070826E305
:10032000036A0B51F2CF0FF3F29E0001E2DE0301EC
:100330000FBFF28E0E6F93988A880C6B0C510708D2
:1003400011E30EAF03D093928A8202D093928A92E5
:10035000939A8A8AD8900E37939A8A9A93988A9811
:100360000C2BECD793928A820B2BD7D70D2BD1D79E
:10037000320E0F6F000145DF03010A076AD7156BC4
:10038000176B166B0001EADE000CEC0ED76E780ED0
:10039000D66E928280B216D01F2A1F3C02D0FE0E6B
:1003A0001F6E1F507D0808E10301096B010E0A6FE3
:1003B00000013CDF010E1D6E1F50060802E2010E17
:1003C0001E6E01D01F6A928680B60BD0212A213C76
:1003D00002D0FE0E216E2150060802E2010E206EB0
:1003E00002D0216A206A928480B40BD0232A233C55
:1003F00002D0FE0E236E2350060802E2010E226E8A
:1004000002D0236A226A928880B812D01A2A1A501F
:10041000100801E21A6A1A50060809E1040E1926AA
:100420001950D00802E2D00E196E010E1C6E01D0D8
:100430001A6A928A80BA12D01B2A1B50200801E245
:100440001B6A1B50060809E1040E195E19500F08BB
:1004500002E3100E196E010E1C6E01D01B6A2652AB
:100460000BE0252A2550130807E2245202E0246AF3
:1004700002D0010E246E256AF2942CEF00F00301E5
:10048000086B0851070811E394928B8207AF03D0E1
:1004900094928B8202D094928B9294948B94D89065
:1004A000073794948B84082BECD794928B9200019D
:1004B000000C0301026B94928B82036B03510708BB
:1004C00011E394948B94000094948B849486000E92
:1004D00082B6010E02130351060802E3D8900237D8
:1004E000032BECD702C301F00001000C0301006BE9
:1004F0000201FF6B03010051070811E30001D9DF7E
:1005000001C001F30301013D01D009D00201FF2B1D
:10051000D8A403D00301002B0201ECD70301013D55
:1005200001D003D0010E016E50D00201FA514009F2
:100530000301026F076F0001A2DFFEC203F3030194
:10054000046B056B066BFEC207F3000198DFFDC26A
:1005500003F3FEC204F30301056B066BFDC207F350
:1005600000018DDFFCC203F3FDC204F3FEC205F3FC
:100570000301066BFCC207F3000181DFFBC207F336
:100580007EDF950E0301076F000179DF0301006B29
:100590000201FF6B03010051070815E3000189DF29
:1005A00001C001F303010151FE0801E10CD001BFBC
:1005B00001D009D00201FF2BD8A403D00301002BE6
:1005C0000201E8D7030101C301F00001000C94907F
:1005D0008B800201D06BD051310808E3FF0E03017C
:1005E000076F00014CDF0201D02BF5D794908B9060
:1005F000FA6BFE6BFD6BFC6BFB6B000177DF02019E
:10060000D02D01D00ED0D03D01D00BD0FA6BFE6BB7
:10061000FD6BFC6BFB6B000169DF01C0D0F2EFD713
:100620000201D02D0CD0010EFA6FFE6BFD6BFC6B3E
:10063000FB6B00015BDF01C0D0F20201F2D7D0C238
:1006400001F0000147EF0BF0186AF2BE188EF29E1F
:10065000640E03010F6F0001D4DD18BEF28E02019B
:10066000D05350E0F2CFD2F2F29E010EA96EA69CBA
:10067000A69EA680A850D2BFF28ED16F0001BF51B6
:100680000201D15D04E10001C05317E00201010E37
:10069000A96EBFC0A8FFA69CA69EA684F2CF00F0BC
:1006A000F29E0F01550EA76EAA0EA76EA682A6B2E5
:1006B000FED7A6940050F2120001F2CFD2F2F29EC1
:1006C000A96AA69CA69EA680A8500201D2BFF28E5F
:1006D000D16F1950D15D15E0A96A19C0A8FFA69C79
:1006E000A69EA684F2CF00F0F29E0F01550EA76ED3
:1006F000AA0EA76EA682A6B2FED7A6940050F2124A
:10070000020115D0010EA96EA86EA69CA69EA68415
:10071000F2CF00F0F29E0F01550EA76EAA0EA76E43
:10072000A682A6B2FED7A6940050F2120201186A61
:10073000F2BE188EF29E640E03010F6F000161DDA0
:1007400018BEF28E939E8A9E186AF2BE188EF29E92
:10075000640E03010F6F000154DD18BEF28E949AEF
:100760008B9A94988B980300000C0201F96BF95155
:1007700063083BE394908B90110EFA6FF4C2FEF283
:10078000F3C2FDF2F2C2FCF2F1C2FBF20001AEDEF6
:1007900001C0F7F20201F75319E1F66BF56BF65160
:1007A000130813E303E1F55187080FE3000181DE2D
:1007B00001C0F8F20201F851FE0803E1000E016EDB
:1007C00016D0F52BD8B4F62BEAD70DD0F751FE088A
:1007D00003E1000E016E0BD094908B800A0E006E28
:1007E000002EFED70000F92BC2D7010E016E0001CA
:1007F000000C5FDE5EDE0201F26BF16BF251070866
:100800000CE3000156DE013C03D0020106D00001DA
:100810000201F12BD8B4F22BF1D70001000C020138
:10082000ED6BE551FE0BEE6FE6C2EFF2E7C2F0F2C0
:10083000E7C2F4F2E6C2F3F2F26FEDC2F1F20001A8
:1008400094DF015201E037D00201E4C2EAF2E5513F
:10085000010BEB6FE96BE86BE95101082AE3EA5100
:10086000E85D20E1EB51E95D1DE1EC6BEC511F0807
:1008700018E3036AEC512A0F016E000E032201C037
:10088000EDF203C0EEF2000114DEEEC2EAFFEDC2AB
:10089000E9FF01C0EFFF0201E82BD8B4E92BEC2BF4
:1008A000E5D703D0000105DE0201E82BD8B4E92B1F
:1008B000D3D700019EDF000C0201F56BF66B010E31
:1008C000F76FDA6AD96A020EFA6FED0EF96F020E4F
:1008D000EA6EF10EE96EFAC2E2FFF9C2E1FFF7C279
:1008E000F8F2D890E550EE02F350F523F450F623D9
:1008F000F82FF7D7F5C2DEFFF6C2F5F2F66BD8B0E7
:10090000F62BF92BD8B4FA2BF72BF7510508DFE1BA
:100910000001000C006A016A026A036A0201E46BCA
:10092000E56BE66BE76BE351E211E111E0112CE0BE
:10093000200EE86FD890DC37DD37DE37DF37E4375D
:10094000E537E637E737E351E75D08E1E251E65D79
:1009500005E1E151E55D02E1E051E45D0FE3E051C5
:10096000E45FE151D8A0E13DE55FE251D8A0E23D6E
:10097000E65FE351D8A0E33DE75FD880003601365B
:1009800002360336E82FD6D7020EEA6EE40EE96E81
:10099000000178EF06F00201E76BE66B010EE56FF0
:1009A000BE0EE46F00013BDF0201DF6BDE6BDD6B2F
:1009B000E26BE16B006A00503224D46F3350DD21CA
:1009C000D56FE151DE21D66FE251DF21D76FD8908C
:1009D000DC6BD435DD6FD535DE6FD635DF6FE76F75
:1009E000DEC2E6F2DDC2E5F2DCC2E4F2000117DFAE
:1009F0000201DF6BDE6BDD6BE26BE16B006A0050C6
:100A00003524D86F3650DD21D96FE151DE21DA6F00
:100A1000E251DF21DB6FD85307E1D951020804E12D
:100A2000DA5302E1DB5303E0010E016E78D137C0E7
:100A3000AAF038C000F0016A026A036A3850D4256F
:100A4000DC6F0150D521DD6F0250D621DE6F0350DF
:100A5000D721DF6FE26BE16BE2C203F0E1C202F08B
:100A6000006A0050DC250001AF6F39500201DD2122
:100A70000001B06F02500201DE210001B16F03508E
:100A80000201DF210001B26F0201DF6BDE6BDD6B63
:100A9000E26BE16BE2C203F0E1C202F0006A0050D7
:100AA0003B240001AB6F3C500201DD210001AC6F23
:100AB00002500201DE210001AD6F03500201DF216F
:100AC0000001AE6F0201DF6BDE6BDD6BE26BE16B91
:100AD000006A00504024D86F4150DD21D96FE151A8
:100AE000DE21DA6FE251DF21DB6FD85309E1D95300
:100AF00007E1DA5305E1DB5303E1010E016E0FD18B
:100B0000DF6BDE6BDD6B3AC0DCF2DFC2F0F2DEC21F
:100B1000EFF2DDC2EEF23AC0EDF2DBC2F4F2DAC27D
:100B2000F3F2D9C2F2F2D8C2F1F20001C5DE0050F0
:100B3000AF25B36F0150B021B46F0250B121B56F32
:100B40000350B221B66FAE310201DB6F0001AD314F
:100B50000201DA6F0001AC310201D96F0001AB3143
:100B60000201D86FDB33DA33D933D833DB33DA33EE
:100B7000D933D833DB33DA33D933D8330F0EDB171D
:100B80000001AB510F0B006E016A026A036A00524A
:100B900006E1015204E1025202E1035209E0010EB2
:100BA0000201D827D8B0D92BD8B4DA2BD8B4DB2B94
:100BB0000201D8510001B325B76F0201D9510001DC
:100BC000B421B86F0201DA510001B521B96F0201F9
:100BD000DB510001B621BA6F0201DF6BDE6BDD6B0A
:100BE000E26BE16B006A00503D24D06F3E50DD2186
:100BF000D16FE151DE21D26FE251DF21D36FD053AB
:100C000058E1D15356E1D25354E1D35352E1D89035
:100C1000DC6BD435DD6FD535DE6FD635DF6F200E5A
:100C2000DC25E06F000EDD21E16F000EDE21E26FBA
:100C3000000EDF21E36FE76FE2C2E6F2E1C2E5F208
:100C4000E0C2E4F20001EBDD0201DF6BDE6BDD6B85
:100C5000E26BE16B2BC001F0006A00502A24E56FC3
:100C60002B50DD21E66FE151DE21E76FE251DF21FC
:100C7000E86FEA6B2CC002F0006A016A0050E525BB
:100C8000EE6F0150E621EF6F2C50E721F06FEA5133
:100C9000E821F16F006A016A026A0050EE25D06F08
:100CA0000150EF21D16F0250F021D26F2D50F12170
:100CB000D36F0001AF510201D05F0001B0510201BA
:100CC000D15B0001B1510201D25B0001B2510201BE
:100CD000D35BD3C2DFF2D2C2DEF2D1C2DDF2D0C228
:100CE000DCF2E36BE26BE16BAAC0E0F2000112D62A
:100CF00003C0D3F202C0D2F201C0D1F200C0D0F2E0
:100D00000201D35305E1D25303E1D1510F0804E2AC
:100D1000000E016E04D003D0010E016E00D0000160
:100D20005DEF0BF00201EC6BD890E66B0001B33580
:100D30000201E76F0001B4350201E86F0001B5352B
:100D40000201E96FE56BE46BE36BE26BE5510001D7
:100D5000AE5DD8A07AD016E10201E4510001AD5D8C
:100D6000D8A073D00FE10201E3510001AC5DD8A01F
:100D70006CD008E1AB510201E25DD8A002D00001C5
:100D800064D00001E9C2F4F2E8C2F3F2E7C2F2F281
:100D9000E6C2F1F2EADC015204E00201ECC201F029
:100DA00057D00201EA6BEA510F083EE3EB6BEB51BF
:100DB0001F0816E3036AEB512A0F016E000E03228F
:100DC00001C0EDF203C0EEF2000159EC02F0EEC2F8
:100DD000EAFFEDC2E9FF01C0EFFF0201EB2BE7D70D
:100DE0002A5201E121D0445202E1455213E02A5037
:100DF000E50810E03550180B0DE132504D080AE1BE
:100E00003350500807E13450330804E1EC2BE12F54
:100E100001D00AD0010EE227D8B0E32BD8B4E42BDE
:100E2000D8B4E52BEA2BBFD70001E3DC2A5201E15D
:100E30000CD00201E15303E1000107D00201020ED0
:100E4000E727000EE823E92381D70201ECC201F075
:100E50000001000C000E016EC250C70B0110C26EE3
:100E6000C284C2B4FED7C3CF27F0C4CF28F0285025
:100E700002082CE303E12750A90828E328500208C0
:100E800018E303E127508A0814E3186AF2BE188EAB
:100E9000F29E0301096B050E0A6F000116EC01F0CA
:100EA00018BEF28E010E0201D06F000124EC03F097
:100EB0000DD0186AF2BE188EF29E0301096B020E65
:100EC0000A6F000116EC01F018BEF28E000C020150
:100ED000E7C2EDF2E851010BEE6FE76BE89100011C
:100EE000CA510201E75D0FE10001CB510201E85D4B
:100EF0000AE10001CC510201E95D05E10001CD519B
:100F00000201EA5D3AE0EAC2F4F2E9C2F3F2E8C2B1
:100F1000F2F2E7C2F1F2000128DC015204E0000E17
:100F2000016E026E4AD00201F06BCE0EEF6FF051EF
:100F3000020818E303E1EF51CD0814E3F0C203F017
:100F4000EF51EF2BD8B4F02BF16F03C0F2F2000198
:100F500059EC02F0F2C2EAFFF1C2E9FF01C0EFFF73
:100F60000201E5D7000145DCEAC2CDF0E9C2CCF0D0
:100F7000E8C2CBF0E7C2CAF00201EEC203F0ED51C5
:100F8000ED2BD8B4EE2BF16FCE0EF125E96E000EED
:100F90000320EA6EEF50EC6BEB6FCE0EED25E96EA1
:100FA000000EEE21EA6EEF50F16F000EEB13F151DF
:100FB000EC13EBC201F0ECC202F0000110EF08F0FC
:100FC000D8900201E76B0001AF350201E86F000124
:100FD000B0350201E96F0001B1350201EA6FEE6B35
:100FE000ED6BD890E135006EE235016EED35026EA5
:100FF000EE35036E0050E725E36F0150E821E46F02
:101000000250E921E56F0350EA21E66FE6C2EAF2F9
:10101000E5C2E9F2E4C2E8F2E3C2E7F2000157D721
:1010200002C0E2F201C0E1F20201E251FE0808E270
:10103000FF0A03E1E151F70803E2FF0EE26FE16FFF
:10104000E1C201F0E2C202F00001000CD0C2E1F204
:1010500069DE01500201D05D03E0090E016E58D235
:10106000D0C2E1F200015EDE0201E46BE36BE26BF1
:10107000E76BE66B47C001F0006A00504624EA6F58
:101080004750E221EB6FE651E321EC6FE751E42199
:10109000ED6FEF6B48C002F0006A016A0050EA256C
:1010A000F36F0150EB21F46F4850EC21F56FEF51D5
:1010B000ED21F66F006A016A026A0050F325000113
:1010C000C26F01500201F4210001C36F02500201FE
:1010D000F5210001C46F49500201F6210001C56FDE
:1010E0000201E26B000E44240001BB6F4550020177
:1010F000E2210001BC6FD890C96BC531C86FC43103
:10110000C76FC331C66FC2C0D9F20001C351010B12
:101110000201DA6F0001BB3D03D0BC3D01D005D018
:10112000BC5308E1BB51010805E3090E016E020141
:10113000EFD10001BCC0E2F2BBC0E1F241DF02C06E
:10114000BEF001C0BDF00201DC6BAAC0DBF2E46BB3
:10115000E36BBCC0E2F2BBC0E1F2020EE15DE56F01
:10116000000EE259E66F000EE359E76F000EE459F6
:10117000E86FAAC000F0016A026A036A03C0ECF2D9
:1011800002C0EBF201C0EAF2AAC0E9F2F06FE7C2D6
:10119000EFF2E6C2EEF2E5C2EDF203C0F4F202C0F5
:1011A000F3F201C0F2F2AAC0F1F200015CEC04F02B
:1011B000B75102010024EA6F0001B8510201012079
:1011C000EB6F0001B95102010220EC6F0001BA512E
:1011D00002010320D890D56BEA35D66FEB35D76F77
:1011E000EC35D86F186AF2BE188EF29E0001C6EC7C
:1011F00000F018BEF28EC65307E1C75305E1C8538D
:1012000003E1C953D8B43ED1D8C2F4F2D7C2F3F245
:10121000D6C2F2F2D5C2F1F2B5EC03F0015204E00D
:10122000090E016E020174D10201D26BD16BD25151
:10123000010824E3938C81ACFDD7000159EC02F046
:1012400001C0DDF293988A880201DE6BDE51070847
:1012500011E3DDAF03D093928A8202D093928A92F7
:10126000939A8A8AD890DD37939A8A9A93988A9823
:10127000DE2BECD7D12BD8B4D22BD9D71E5238E0E5
:10128000938C81ACFDD7186AF2BE188EF29E010EC7
:101290000301096F0A6F000116EC01F018BEF28E0F
:1012A000928280A2FDD71D5206E0010E016E02015E
:1012B0002FD11ED000011E6A010E266E1E5208E1BB
:1012C000245203E0949A8B8A02D0949A8B9AF6D790
:1012D000949A8B8A928280B202D01E6AFBD7266AC9
:1012E000949A8B8A1D5205E0010E016E020110D105
:1012F0000001F29CF29EF2BEFDD71C521FE00201DB
:10130000E26B19C0E1F219C0E4F2E36B036A195011
:10131000E311E56F03501910E66F186AF2BE188EDC
:10132000F29E0B0E0301156FE6C217F3E5C216F32A
:101330000001AEEC00F018BEF28E1C6A1D5205E0F2
:10134000010E016E0201E4D00001205208E0938CEE
:1013500081ACFDD7020E016E0201DAD000012252EB
:1013600008E0938C81ACFDD7030E016E0201D0D052
:101370000001C00EF212FF0EC627D8A0C727D8A0C2
:10138000C827D8A0C9270201DB51D8B4DC07DB2F5E
:1013900002D0DC5306E0020ED627000ED723D82356
:1013A0006FD00001BD530CE1BE530AE1BCC0E2F2B4
:1013B000BBC0E1F205DE02C0BCF001C0BBF006D04C
:1013C000BEC0BCF0BDC0BBF0BE6BBD6BBB3D03D0AF
:1013D000BC3D01D005D0BC5304E1BB51010801E381
:1013E00051D00201E46BE36BBCC0E2F2BBC0E1F29E
:1013F000020EE15DE56F000EE259E66F000EE35963
:10140000E76F000EE459E86FAAC000F0016A026AB3
:10141000036A03C0ECF202C0EBF201C0EAF2AAC018
:10142000E9F2F06FE7C2EFF2E6C2EEF2E5C2EDF2EA
:1014300003C0F4F202C0F3F201C0F2F2AAC0F1F26A
:1014400000015CEC04F0B75102010024EA6F0001D6
:10145000B85102010120EB6F0001B95102010220D5
:10146000EC6F0001BA5102010320D890D56BEA3528
:10147000D66FEB35D76FEC35D86FDC6BAAC0DBF2DB
:101480000001B9D60201D95302E1DA533FE0D8C2D4
:10149000F4F2D7C2F3F2D6C2F2F2D5C2F1F20001F1
:1014A000B5EC03F0015204E0090E016E020130D0E8
:1014B0000201D26BD16BD251DA5D28E303E1D9513D
:1014C000D15D24E2938C81ACFDD7000159EC02F090
:1014D00001C0DFF293988A880201E06BE0510708AF
:1014E00011E3DFAF03D093928A8202D093928A9263
:1014F000939A8A8AD890DF37939A8A9A93988A988F
:10150000E02BECD7D12BD8B4D22BD5D7000E016E5F
:101510000001D7EF0BF0F86AD09E0D8EEA6AE96AF7
:10152000C180C182C184C196926A896A936A8A6ABB
:10153000946A170E8B6EC190C182C184C186C18C22
:10154000C29CC28EC18EC2801F0E926E400E936EE0
:10155000080E946E939E8A9E296A94988B88949A1A
:101560008B8A939E8A8E928280A2FDD7928680B6C5
:1015700002D0010E296E928680A6FDD71A6A1B6AD8
:101580001C6A1D6A1E6A1F6A206A216A226A236A0F
:10159000246A256A266A830ED56EEC0ED76E780E05
:1015A000D66EF28AC00EF212F2CFD0F2F29EA96A83
:1015B000A69CA69EA680A8500201D0BFF28E196EEE
:1015C000193C02D0300E196E1950800802E2600EEC
:1015D000196EF29CF29EF2BEFDD7186AF2BE188E0A
:1015E000F29E0001C6EC00F018BEF28EC00EF212A0
:1015F000186AF2BE188EF29EFA0E03010F6F0001F8
:1016000001EC01F018BEF28EF2CFD0F2F29E010E84
:10161000A96EA69CA69EA680A8500201D0BFF28EFD
:101620000001C06BBF6F295210E0C06B010EBF6F8D
:10163000186AF2BE188EF29E010E0301096F0A6F3E
:10164000000116EC01F018BEF28E186AF2BE188E78
:10165000F29E010E0301096F0A6F000116EC01F002
:1016600018BEF28E020E0201D06F186AF2BE188EFA
:10167000F29EFA0E03010F6F000101EC01F018BE9B
:10168000F28E0201D02FF1D70001E7EF02F0013C0A
:1016900012D0186AF2BE188EF29E0301096B080E72
:1016A0000A6F000116EC01F018BEF28E0201D06B39
:1016B000000124EC03F0CBEF04F0015213E0186AB0
:1016C000F2BE188EF29E010E0301096F080E0A6F1A
:1016D000000116EC01F018BEF28E0201D06B000181
:1016E00024EC03F0FF0E0201E16F000192EC06F022
:1016F00001C0C1F0C15313E1186AF2BE188EF29E08
:10170000010E0301096F040E0A6F000116EC01F0CF
:1017100018BEF28E0201D06B000124EC03F092821D
:1017200080B202D01E6AFBD71D5206E0010E0201F4
:10173000D06F000124EC03F0020E0201D06F186A92
:10174000F2BE188EF29EFA0E03010F6F000101EC3B
:1017500001F018BEF28E0201D02FF1D7928280B232
:1017600002D01E6AFBD71D5205E0010ED06F0001AA
:1017700024EC03F000012AEC07F01D5206E0010EF4
:101780000201D06F000124EC03F0C05303E1BF510C
:10179000C15D03E2C06B010EBF6FBF5305E1C053D3
:1017A00003E1C06BC1C0BFF0BFC0D0F24FD401C0D5
:1017B000CEF20201CE2D06D0010ED06F000124EC36
:1017C00003F00201CE51020817E1186AF2BE188E2A
:1017D000F29E010E0301096F0A6F000116EC01F081
:1017E00018BEF28EBF2BD8B4C02B206A928680B66A
:1017F00002D0206AFBD70201CE51030818E1186A13
:10180000F2BE188EF29E010E0301096F0A6F0001ED
:1018100016EC01F018BEF28EBF51D8B4C007BF0756
:10182000226A928480B402D0226AFBD70201CE5190
:10183000090826E1CF6BCF5103081DE3186AF2BEF9
:10184000188EF29E0301096B010E0A6F000116EC5F
:1018500001F018BEF28E186AF2BE188EF29E010ECA
:101860000301096F0A6F000116EC01F018BEF28E39
:101870000201CF2BE0D7D06B000124EC03F0020172
:10188000CE5304E10001BF2BD8B4C02B00012AECD9
:0618900007F073D703000E
:020000040030CA
:0E00000000060E0E000080000FC00FE00F4043
:00000001FF
